:020000040000FA
:020000007E2858
:08000800F000030E8301F1007A
:100010000A08F2008A0183130408F30083160C1DFA
:10002000132883121528831229280C1D29280C1146
:10003000831698160C118312B2010130A100A2019F
:1000400020140230A400A40B232883160C1683125C
:100050000E2883160C1C2E28831230288312452864
:100060000C1C45288316981C3328831207140000A3
:10007000071090308E00E8308F000C100C118316A2
:1000800098120C100C1583120E2883160C1E4A2889
:1000900083124C28831275280C1E75288316181499
:1000A0008312201C572820102C0899000E282B089A
:1000B0002202A3002A082102031CA303A31B672812
:1000C00033303207840000089900B20A692803011E
:1000D0009900A10A0319A20A3208043A031D0E2846
:1000E00083160C140C1283120E28730884007208F5
:1000F0008A00710E8300F00E700E090085018601E2
:10010000870183163F3085008F308600F0308700EE
:100110008312061786160616AD01861B2D140613CC
:10012000000006090F39A50006178612000006090F
:100130000F39A60086160612000006090F39A7001F
:1001400006161521A9080319B3282908013C031C28
:10015000AE282808FD3C031CB028B8280130A900AF
:10016000FD30A800B828A808031DB8280130A80051
:100170002808AA002908AB000030AC00B2013330D7
:10018000320784008001B20A3208043A031DBF28F6
:1001900083160430990018151812831298178316C5
:1001A0001817981683129001101497019715971439
:1001B00040309500EA3096000C140C1183160C1494
:1001C0000C118C120C1283128B010B178B178316D8
:1001D00002309F0083129F019F171F14AF0133301D
:1001E00084008715000903198711C7309F05031084
:1001F000AF0DAF0D2F0D9F040310AF0CAF0C2130CE
:10020000AE00AE0B01291F151F19042933302F072B
:1002100084002D180D291E080E291E098000AF0A22
:100220002F08043A031DF528EE28A9012508A80087
:1002300021212608A80721212708A8070318A90AB1
:1002400008002808B0002908B1000310A80DA90D66
:100250000310A80DA90D3008A807031C3029A90A0E
:0C0260003108A9070310A80DA90D080023
:02400E00723FFF
:00000001FF
